:1000000054EF06F00000000000EF00F000000000D8
:0A0010000000000000000000F3D71C
:10001C00160E0C6E6C0E0D6E0D2EFED70C2EFCD724
:04002C0000001200BE
:0E003000310E0D6E0D2EFED7000000001200E6
:08003E000000000000001200A8
:100046000101C3BF02D0819E01D0818EC3BD02D003
:10005600819C01D0818CC3BB02D0819A01D0818A58
:10006600C3B902D0819801D08188AEB102D0818413
:1000760001D081948186E0DF8196C3B702D0819E4C
:1000860001D0818EC3B502D0819C01D0818CC3B3CF
:1000960002D0819A01D0818AC3B102D0819801D061
:1000A6008188AEB102D0818401D081948186C4DF7B
:0E00B6008196AEA102D0AFDF01D0B7DF1200FD
:1000C4000FEE81F0EF50EFCF00F0009200C0EFFF91
:0200D400120018
:1000D6000FEE81F0EF50EFCF00F0009000C0EFFF81
:0200E600120006
:0E00E8000101AE91C2C1C3F1AADFAE811200C8
:1000F600086A096A100E0C6E013408360936045077
:10010600085E0550D8A0053C095ED8B007D004505B
:1001160008260550D8B0053C0926D8900036013689
:060126000C2EEAD71200C6
:10012C0010D0800E0101BB6F1AD0C00EBB6F17D060
:10013C00940EBB6F14D0D40EBB6F11D0800EBB6F5E
:10014C000ED00101BB51010AECE0BB51020AEDE0FB
:10015C00BB51030AEDE0BB51040AEDE0EFD7BC053F
:10016C00006EBB51002600C0BBF100C0C3F165DFBF
:10017C00AE91BF6BBF51BD25E96E000EBE21EA6E7C
:10018C00EE520BE0BF51BD25E96E000EBE21EA6EAA
:0E019C00EECFC2F1A3DFBF2BEDD7AE81120074
:1001AA000101BF6B050EBF5D0AE2BF51BD25E16EBD
:1001BA00000EBE21E26E200EE66EBF2BF3D7BF51B2
:1001CA00BD25E16E000EBE21E26EE66ABF07BF5191
:1001DA00BD25C06F000EBE21C16F0A0E046E000E4F
:1001EA00056EBBC100F0BCC101F080DF08C000F0A1
:1001FA0009C001F0300E0026C0C1E1FFC1C1E2FF13
:10020A0000C0E6FF0A0E046E000E056EBBC100F0C8
:10021A00BCC101F06BDF00C0BBF101C0BCF1000E34
:10022A00011802E1000E001801E102D0BF07CFD782
:02023A001200B0
:10023C00010E0101BE6F000EBF6F800EBC6F000E71
:10024C00BD6FBC51BD1123E0F4DEF3DEF2DEF1DE56
:10025C0033DF9392EEDEEDDEBC51BB15006E000E6B
:10026C00BD15016E0050011002E0938002D02DDF0D
:10027C009390DFDEDEDE9382AE9381B204D0AEA328
:10028C0001D001D0FAD7BD33BC33BD9FDAD7BE6BDA
:10029C00BF6BCFDECEDE10DF9392CBDECADE938057
:1002AC00C8DEC7DEC6DEC5DE9382AE9381B204D053
:1002BC00AEA301D001D0FAD7BE6BBF6BBADEB9DEEC
:1002CC0081B0BE81B6DEB5DEB4DEB3DEB2DEB1DE49
:1002DC00B0DEAFDEAEDEADDEACDEABDEAADEA9DEBE
:1002EC00A8DEA7DEE9DE9392F0DE9390BEC100F0AB
:0202FC001200EE
:1002FE000101BD6BBE6B800EBF6F000EC06FBF5194
:10030E00C0111BE095DE94DE938092DE91DE938227
:10031E00AE9381B204D0AEA301D001D0FAD781A0A2
:10032E0004D0BF51BD13C051BE1382DE81DEC3DEC9
:10033E009392C033BF33C09FE2D7938079DE78DECD
:10034E00BB51BC1102E0C0DE939072DE71DE93826F
:10035E00AE9381B204D0AEA301D001D0FAD768DE3D
:10036E0067DEA9DE939264DE63DEAEDE9390BDC1DE
:04037E0000F0120079
:10038200A9DE93905BDE5ADE93820101AE9381B2C5
:1003920004D0AEA301D001D0FAD750DE4FDE4EDE3C
:1003A2004DDE4CDE4BDE4ADE49DE938047DE46DE22
:0203B200120037
:1003B400938043DE42DE938240DE3FDE8ADE93900A
:0A03C4003CDE3BDE7DDE939212006A
:1003CE0010D0800E0101BB6F1AD0C00EBB6F17D0BC
:1003DE00940EBB6F14D0D40EBB6F11D0800EBB6FBA
:1003EE000ED00101BB51010AECE0BB51020AEDE057
:1003FE00BB51030AEDE0BB51040AEDE0EFD7BC059B
:10040E00006EBB51002600C0BBF1AE8100C0C3F12F
:0E041E0013DEAE91BDC1C3F10FDEAE81120040
:10042C00086A080E0C6E003408360450085ED8B00A
:0E043C0002D00826D89000360C2EF5D71200FC
:10044A000900F5CFE6FF0006FBE10106F9E112001B
:10045A00A6A202D00000FCD7A69CB1C1A9FFB2C1D6
:10046A00A8FFA69EA684F2CF00F0F29E550EA76EB4
:10047A00AA0EA76EA68200BE02D0F29E01D0F28E0C
:04048A00A694120022
:10048E00939693949398939A939C939E819681942A
:10049E00819E819C819A8198BADDB9DDB8DD818A11
:1004AE0081888186C5DD8196B2DD8186C1DD81962A
:1004BE00AEDD8186BDDD8196AADD81988186B8DDAF
:1004CE008196A5DD8186B4DD8196819A818E8186A5
:1004DE00AFDD81969CDD819E81888186A9DD819626
:1004EE0081988186A5DD819692DD8186A1DD81963A
:1004FE00818881869DDD81968ADD8198818698DD51
:10050E008196818E818C818A8188818691DD81960A
:08051E007EDD0101AE81120037
:1005260082AC27D0000E1C1802E1060E1B1821E033
:100536001D0E1B24E16E000E1C20E26E300EE66ED0
:100546001B4A1C2A300E0101C26FCBDD040E0B6E56
:10055600CF0E0C6E010E0D6E0D2EFED70C2EFCD797
:100566000B2EFAD700000000176A186A196A1A6A71
:10057600C6D182A027D0000E1C1802E1060E1B1859
:1005860021E001011D0E1B24E16E000E1C20E26E0F
:10059600310EE66E1B4A1C2A310EC26FA2DD040E16
:1005A6000B6ECF0E0C6E010E0D6E0D2EFED70C2EA1
:1005B600FCD70B2EFAD700000000176A186A196AD2
:1005C6001A6A9DD182A227D0000E1C1802E1060EDF
:1005D6001B1821E001011D0E1B24E16E000E1C20DC
:1005E600E26E320EE66E1B4A1C2A320EC26F79DDAF
:1005F600040E0B6ECF0E0C6E010E0D6E0D2EFED779
:100606000C2EFCD70B2EFAD700000000176A186ACA
:10061600196A1A6A74D182A427D0000E1C1802E146
:10062600060E1B1821E001011D0E1B24E16E000EB3
:100636001C20E26E330EE66E1B4A1C2A330EC26F76
:1006460050DD040E0B6ECF0E0C6E010E0D6E0D2ED0
:10065600FED70C2EFCD70B2EFAD700000000176A27
:10066600186A196A1A6A4BD183A027D0000E1C1883
:1006760002E1060E1B1821E001011D0E1B24E16E8E
:10068600000E1C20E26E340EE66E1B4A1C2A340E47
:10069600C26F27DD040E0B6ECF0E0C6E010E0D6EB3
:1006A6000D2EFED70C2EFCD70B2EFAD7000000001D
:1006B600176A186A196A1A6A22D183AE27D0000E01
:1006C6001C1802E1060E1B1821E001011D0E1B2459
:1006D600E16E000E1C20E26E350EE66E1B4A1C2AE9
:1006E600350EC26FFEDC040E0B6ECF0E0C6E010EC5
:1006F6000D6E0D2EFED70C2EFCD70B2EFAD7000052
:100706000000176A186A196A1A6AF9D083AC27D0EA
:10071600000E1C1802E1060E1B1821E001011D0E39
:100726001B24E16E000E1C20E26E360EE66E1B4A9E
:100736001C2A360EC26FD5DC040E0B6ECF0E0C6E65
:10074600010E0D6E0D2EFED70C2EFCD70B2EFAD7F2
:1007560000000000176A186A196A1A6AD0D083AABC
:1007660027D0000E1C1802E1060E1B1821E001011D
:100776001D0E1B24E16E000E1C20E26E370EE66E87
:100786001B4A1C2A370EC26FACDC040E0B6ECF0E52
:100796000C6E010E0D6E0D2EFED70C2EFCD70B2EF9
:1007A600FAD700000000176A186A196A1A6AA7D0F1
:1007B60083A827D0000E1C1802E1060E1B1821E0A4
:1007C60001011D0E1B24E16E000E1C20E26E380E88
:1007D600E66E1B4A1C2A380EC26F83DC040E0B6EB3
:1007E600CF0E0C6E010E0D6E0D2EFED70C2EFCD705
:1007F6000B2EFAD700000000176A186A196A1A6ADF
:100806007ED082AE27D0000E1C1802E1060E1B1801
:1008160021E001011D0E1B24E16E000E1C20E26E7C
:10082600390EE66E1B4A1C2A390EC26F5ADC040EBC
:100836000B6ECF0E0C6E010E0D6E0D2EFED70C2E0E
:10084600FCD70B2EFAD700000000176A186A196A3F
:100856001A6A55D082A853D0000E1C1802E1060E63
:100866001B184DE001011B6A1C6A010EC36F23ECC5
:1008760000F0000E0001D61902E1000ED51913E1B1
:10088600010E0101BB6F010EBC6FB30EBD6F000EF2
:10089600BE6F49DC020EBB6F010EBC6FC20EBD6F90
:1008A600000EBE6F40DC000E0001D61902E1010EFB
:1008B600D51913E1010E0101BB6F010EBC6FED0EE0
:1008C600BD6F000EBE6F2FDC020EBB6F010EBC6F3C
:1008D600FE0EBD6F000EBE6F26DC040E0B6ECF0E35
:1008E6000C6E010E0D6E0D2EFED70C2EFCD70B2EA8
:1008F600FAD700000000176A186A196A1A6A120005
:10090600938293800101AE9381B204D0AEA301D04D
:0609160001D0FAD7120027
:10091C00010E0101BB6F060EBC6F0A0E046EAAC15C
:10092C0000F07EDD300E0024BD6F4BDD010EBB6F81
:10093C00070EBC6F0A0E046EAAC100F071DD08C070
:10094C0000F0300E0024BD6F3CDD010EBB6F090EB4
:10095C00BC6F0A0E046EA8C100F062DD300E0024DC
:10096C00BD6F2FDD010EBB6F0A0EBC6F0A0E046E3D
:10097C00A8C100F055DD08C000F0300E0024BD6F9A
:10098C0020DD010EBB6F0F0EBC6F350EAD25BD6F9C
:10099C0018DD020EBB6F060EBC6F0A0E046EA9C1E9
:1009AC0000F03EDD300E0024BD6F0BDD020EBB6F80
:1009BC00070EBC6F0A0E046EA9C100F031DD08C031
:1009CC0000F0300E0024BD6FFCDC020EBB6F090E74
:1009DC00BC6F0A0E046EACC100F022DD300E002498
:1009EC00BD6FEFDC020EBB6F0A0EBC6F0A0E046EFD
:1009FC00ACC100F015DD08C000F0300E0024BD6F56
:100A0C00E0DC020EBB6F0C0EBC6F0A0E046EABC1A9
:100A1C0000F006DD300E0024BD6FD3DC020EBB6F80
:100A2C000D0EBC6F0A0E046EABC100F0F9DC08C0F1
:0C0A3C0000F0300E0024BD6FC4DC12007E
:100A48000101B76BB86BB1C1B9F1B2C1BAF1800E8F
:100A5800B219006E800E005C02E1000EB15D0BE27F
:100A6800010EB76F000EB86FB1510008B96FB2C16F
:100A7800BAF1000EBA57B9C1BBF1BAC1BCF1B3C1E2
:100A8800BDF1B4C1BEF1D5EC00F0060EB56F000E95
:100A9800B66F000E006EB651005C02E1B551000859
:100AA80019E2B551B325E16EB651B421E26E010EDB
:100AB800B55D006E000EB659016E0050B325E96EA3
:100AC8000150B421EA6EEECFE6FF010EB55F000ECD
:100AD800B65BDFD7B3C1E1FFB4C1E2FF200EE66E1B
:100AE800B751B8111AE0B56BB66BB551B325E96EBD
:100AF800B651B421EA6EEE50200A03E1B54BB62B8D
:100B0800F4D7010EB55F000EB65BB551B325E16EA3
:0C0B1800B651B421E26E2D0EE66E120004
:100B2400F00E0101AB15026E02C000F00032009E0F
:100B34000032009E0032009E0032009E0A0E000227
:100B4400F3CF01F00F0EAB15006E00500124AB6F14
:100B5400F00EAC15026E02C000F00032009E0032AE
:100B6400009E0032009E0032009E0A0E0002F3CF67
:100B740001F00F0EAC15006E00500124AC6FF00EA6
:100B8400A915026E02C000F00032009E0032009EE1
:100B94000032009E0032009E0A0E0002F3CF01F0E4
:100BA4000F0EA915006E00500124A96FC00EAA15DE
:100BB400AD6F060E006E005004E0AD33AD9FFF0F25
:100BC400FBD7300EAA15026E02C000F00032009E60
:100BD4000032009E0032009E0032009E0A0E000287
:100BE400F3CF01F00F0EAA15006E00500124AA6F76
:100BF400100EA815026E02C000F00032009E0032F2
:100C0400009E0032009E0032009E0A0E0002F3CFC6
:100C140001F00F0EA815006E00500124A86F1200F9
:100C2400A69CB1C1A9FFA69EA680A8CF00F0120081
:100C3400DAEC01F0A00E0101BB6F1EEC01F0020E14
:100C4400BB6F1EEC01F0DAEC01F0A10EBB6F1EECE1
:100C540001F0010EBB6F000EBC6F7FEC01F000C011
:100C6400ABF1010EBB6F000EBC6F7FEC01F000C056
:100C7400ACF1010EBB6F000EBC6F7FEC01F000C045
:100C8400A9F1010EBB6F000EBC6F7FEC01F000C038
:100C9400AAF1BB6BBC6B7FEC01F000C0A8F1C1EC06
:040CA40001F0120049
:100CA80026EC0CF00F0EC16E070EB4127F0ED36E39
:100CB800936AFF0E8A6EFF0E8B6E929492966D96D3
:100CC8006F86F90E956E010E0101B16F310EB26F8C
:100CD8002DEC02F0020E0101B16F340EB26F2DEC53
:100CE80002F0030E0101B16F300EB26F2DEC02F06D
:100CF800040E0101B16F350EB26F2DEC02F0050E36
:100D08000101B16F390EB26F2DEC02F0060E010130
:100D1800B16F350EB26F2DEC02F08096809447ECDF
:100D280002F0EDDD010E0101C36F23EC00F00C0EA3
:100D3800C36F23EC00F0010EBB6F010EBC6F870E72
:100D4800BD6F000EBE6F96EC00F0070E0B6E170E0F
:100D58000C6E6A0E0D6E01010D2EFDD70C2EFBD701
:100D68000B2EF9D70000010EBB6F010EBC6F790E78
:100D7800BD6F000EBE6F96EC00F0070E0B6E170EDF
:100D88000C6E6A0E0D6E0D2EFED70C2EFCD70B2E98
:100D9800FAD70000010EBB6F010EBC6FA40EBD6F29
:100DA800000EBE6F96EC00F0070E0B6E170E0C6E61
:100DB8006A0E0D6E0D2EFED70C2EFCD70B2EFAD711
:100DC8000000010EBB6F010EBC6F940EBD6F000ECC
:100DD800BE6F96EC00F0070E0B6E170E0C6E6A0EC7
:100DE8000D6E0D2EFED70C2EFCD70B2EFAD7000059
:100DF800010EBB6F010EBC6F650EBD6F000EBE6F9E
:100E080096EC00F0070E0B6E170E0C6E6A0E0D6E48
:100E18000D2EFED70C2EFCD70B2EFAD70000010E94
:100E2800C36F23EC00F0010EBB6F060EBC6F5D0EA6
:100E3800BD6F000EBE6F96EC00F0080E0B6E9D0E97
:100E48000C6E050E0D6E0D2EFED70C2EFCD70B2E3C
:100E5800FAD700000000010EC36F23EC00F0010E6A
:100E6800BB6F010EBC6FB30EBD6F000EBE6F96EC6C
:100E780000F0070E0B6E170E0C6E6A0E0D6E0D2E1F
:100E8800FED70C2EFCD70B2EFAD70000020EBB6F34
:100E9800010EBC6F780EBD6F000EBE6F96EC00F0B1
:100EA80093EC02F0010E0101B16FB8DE1D5000187D
:100EB80036E1020EB16FB2DE1E50001830E1030EAB
:100EC800B16FACDE1F5000182AE1040EB16FA6DE28
:100ED8002050001824E1050EB16FA0DE2150001843
:100EE8001EE1060EB16F9ADE2250001818E1000EBE
:100EF8001C1802E1060E1B1812E1000E00017719FA
:100F080002E1000E76190BE1010E0101BB6F010E23
:100F1800BC6FD70EBD6F000EBE6F96EC00F082AAB4
:100F2800ACD00101010EB16F79DE1D500018D8A4B4
:100F3800A4D0020EB16F72DE1E500018D8A49DD046
:100F4800030EB16F6BDE1F500018D8A496D0040EA4
:100F5800B16F64DE20500018D8A48FD0050EB16F91
:100F68005DDE21500018D8A488D0060EB16F56DE79
:100F780022500018D8A481D0000E1C1802E1060ED9
:100F88001B18D8A47AD0000E0001771902E1000ED0
:100F9800761973E1010E0101C36F23EC00F0010E15
:100FA800BB6F010EBC6FC30EBD6F000EBE6F96EC1B
:100FB80000F0110E0B6EBE0E0C6EA90E0D6E0D2EEE
:100FC800FED70C2EFCD70B2EFAD700000000808429
:100FD8001B6A1C6A156A166A010EBB6F010EBC6F8C
:100FE8004C0EBD6F000EBE6F96EC00F0020EBB6F8C
:100FF800010EBC6F3E0EBD6F000EBE6F96EC00F08A
:10100800030E0A6EDB0E0B6E840E0C6E110E0D6E47
:101018000D2EFED70C2EFCD70B2EFAD70A2EF8D79A
:10102800000000008094300E226E300E216E300ECB
:10103800206E300E1F6E300E1E6E300E1D6E010EAD
:10104800C36F23EC00F0010EBB6F010EBC6F260EC0
:10105800BD6F000EBE6F96EC00F0246A256A270E5D
:101068000B6E0D0E0C6E260E0D6E0D2EFED70C2E71
:10107800FCD70B2EFAD70000EED683A657D0000E69
:10108800251802E1000E241851E10101010EBB6F81
:10109800010EBC6F380EBD6F000EBE6F96EC00F0EF
:1010A800010EBB6F080EBC6F2F0EBD6FE7EC01F091
:1010B800010EBB6F0B0EBC6F2F0EBD6FE7EC01F07E
:1010C800020EBB6F010EBC6F320EBD6F000EBE6FFD
:1010D80096EC00F0020EBB6F080EBC6F3A0EBD6FA7
:1010E800E7EC01F0020EBB6F0B0EBC6F3A0EBD6F42
:1010F800E7EC01F0010EBB6F0C0EBC6F860EBD6FE6
:10110800010EBE6F96EC00F0846B856B000E006ECE
:101118008551005C02E184513C0807E387DDFEDC71
:101128008EEC04F0844B852BF1D795D682AAB5D0E6
:10113800000E161802E1030E1518D8B4AED0000E32
:10114800161802E1040E1518D8B4A7D00101010E33
:10115800C36F23EC00F0010EBB6F010EBC6FB30E22
:10116800BD6F000EBE6F96EC00F0020EBB6F010E55
:10117800BC6F8A0EBD6F010EBE6F96EC00F0100EAC
:101188000B6E390E0C6E0D0E0D6E0D2EFED70C2E3D
:10119800FCD70B2EFAD700000000010E0001766F75
:1011A800000E776F010E0101C36F23EC00F0000EF3
:1011B800161802E1000E15180DE1010EBB6F010EA5
:1011C800BC6F6A0EBD6F010EBE6F96EC00F0154A3B
:1011D800162A2DD0000E161802E1010E15180DE181
:1011E800010EBB6F010EBC6F770EBD6F010EBE6F97
:1011F80096EC00F0154A162A1AD0000E161802E1CD
:10120800020E151814E10101010EBB6F010EBC6F2F
:101218005E0EBD6F010EBE6F96EC00F0030E156EEC
:10122800000E166E010E0001D56F000ED66F100E5F
:101238000B6E390E0C6E0D0E0D6E0D2EFED70C2E8C
:10124800FCD70B2EFAD700000000010E0101C36F76
:1012580023EC00F0010EBB6F010EBC6FB30EBD6F27
:10126800000EBE6F96EC00F0070E0B6E170E0C6E9C
:101278006A0E0D6E0D2EFED70C2EFCD70B2EFAD74C
:101288000000020EBB6F010EBC6F4C0EBD6F010E4D
:10129800BE6F96EC00F01B6A1C6A82AA74D0000E1E
:1012A800161802E1030E15186EE1000E00017719F9
:1012B80002E1010E761967E1010E0101C36F23EC0B
:1012C80000F0010EBB6F010EBC6FB30EBD6F000EB8
:1012D800BE6F96EC00F0020EBB6F010EBC6F8A0E5B
:1012E800BD6F010EBE6F96EC00F080861B6A1C6A0B
:1012F800100E0B6E390E0C6E0D0E0D6E0D2EFED7E8
:101308000C2EFCD70B2EFAD700000000010EC36F7D
:1013180023EC00F0010EBB6F010EBC6F4D0EBD6FCC
:10132800010EBE6F96EC00F0100E0B6E390E0C6EAF
:101338000D0E0D6E0D2EFED70C2EFCD70B2EFAD7E8
:1013480000000000010EC36F23EC00F0010EBB6F1C
:10135800010EBC6FED0EBD6F000EBE6F96EC00F077
:10136800020EBB6F010EBC6F9C0EBD6F010EBE6FEF
:1013780096EC00F0020E0001766F000E776F010EFA
:10138800246E000E256E82AA76D0000E161802E191
:10139800030E1518D8A46FD01D50310A6CE11E50E9
:1013A800390A69E11F50380A66E12050340A63E1BE
:1013B800010E0101C36F23EC00F08096010EBB6F94
:1013C800010EBC6F9D0EBD6F010EBE6F96EC00F056
:1013D800100E0B6E390E0C6E0D0E0D6E0D2EFED707
:1013E8000C2EFCD70B2EFAD7000000001B6A1C6AD3
:1013F800010EC36F23EC00F0010EBB6F010EBC6F32
:101408003C0EBD6F010EBE6F96EC00F0010EC36F6F
:1014180023EC00F0010EBB6F010EBC6F3C0EBD6FDC
:10142800010EBE6F96EC00F0000E2A1902E1000EC4
:1014380029190AE1020EBB6F010EBC6F2B0EBD6F9E
:10144800010EBE6F96EC00F0000E2A1902E1010EA3
:1014580029190AE1020EBB6F010EBC6F2C0EBD6F7D
:10146800010EBE6F96EC00F0040E156E000E166E9F
:101478000001766B776B82AA53D0000E161802E132
:10148800040E15184DE1010E0101B16F1DC0B2F136
:101498002DEC02F0020E0101B16F1EC0B2F12DEC6D
:1014A80002F0030E0101B16F1FC0B2F12DEC02F082
:1014B800040E0101B16F20C0B2F12DEC02F0050E4F
:1014C8000101B16F21C0B2F12DEC02F0060E01014D
:1014D800B16F22C0B2F12DEC02F0010E0101C36F11
:1014E80023EC00F0010EBB6F010EBC6F220EBD6F26
:1014F800010EBE6F96EC00F0080E0B6E9D0E0C6E82
:10150800050E0D6E0D2EFED70C2EFCD70B2EFAD71E
:1015180000000000156A166A010EC36F23EC00F084
:1015280082AAC3D0000E161802E1030E1518D8A41B
:10153800BCD0000E0001771902E1020E7619D8A47A
:10154800B4D0000E251802E1010E2418D8A4ADD09D
:10155800010E0101BB6F010EBC6FED0EBD6F000ED9
:10156800BE6F96EC00F0020EBB6F010EBC6FFF0E53
:10157800BD6F000EBE6F96EC00F0060E1B6E000EDF
:101588001C6E020EBB6F010EBC6F000EBD6F010E0C
:10159800BE6F96EC00F01F0E0B6E710E0C6E1E0ED9
:1015A8000D6E0D2EFED70C2EFCD70B2EFAD7000091
:1015B800010EC36F23EC00F0010EBB6F010EBC6F70
:1015C800110EBD6F010EBE6F96EC00F0020EBB6FE0
:1015D800010EBC6F2F0EBD6F010EBE6F96EC00F0B2
:1015E800010E296F000E2A6F02D0AF4BB02BAF6BE4
:1015F800B06B000E006EB051005C02E1AF513C08C8
:1016080029E33AC1B1F13BC1B2F12E0EB36F010E1D
:10161800B46F24EC05F0020EBB6F0A0EBC6F2E0EE1
:10162800BD6F010EBE6F96EC00F0010E3A5F000E22
:101638003B5B0F0E0B6E140E0C6ED90E0D6E0D2E3D
:10164800FED70C2EFCD70B2EFAD700000000AF4BAC
:10165800B02BCFD7000E006EB051005C02E1AF5145
:101668003C08C3E23C0E3A6F000E3B6F010EC36F9D
:1016780023EC00F0010EBB6F010EBC6FED0EBD6FC9
:10168800000EBE6F96EC00F0020EBB6F010EBC6F31
:101698002D0EBD6F010EBE6F96EC00F0020E00011C
:1016A800766F000E776F1B6A1C6A54EF07F0FFD73E
:10184C0010EE15F0930E006E020E016EB80EF66ED1
:0E185C00160EF76E000EF86E25EC02F012006C
:0216B800000030
:0216BA0000002E
:0216BC0000002C
:0216BE0000002A
:0716C0000000000000000023
:0216C700000021
:0C16C9004761746520436C6F736564001A
:0616D50054696D653A0046
:0616DB00446174653A0051
:0E16E10031206D696E20617070726F782E007E
:1016EF0047617465206F70656E656420666F722048
:0116FF0000EA
:0817000057656C636F6D650015
:10170800496E697469616C697A696E672E2E2E2E2E
:0117180000D0
:021719000000CE
:01171B0000CD
:0E171C00496E697469616C697A696E672E00A6
:0D172A00496E697469616C697A696E6700C7
:10173700496E697469616C697A696E672E2E2E002D
:0F174700496E697469616C697A696E672E2E004C
:0F175600456E7465722070696E636F64653A004A
:011765000083
:1017660041636365737320417070726F7665642E92
:02177600000071
:0217780000006F
:10177A005072657373204F4B202020202020202098
:06178A00202020200000D9
:10179000456E74657220416C742E20636F64653AE7
:0117A0000048
:0117A1000047
:0117A2000046
:1017A30057726F6E6720416C742E20636F646500FF
:0117B3000035
:1017B4005761697420666F722036302073656373D5
:0117C4000024
:0717C50053617665642E00FC
:0217CC0000001B
:0117CE00001A
:0117CF000019
:0117D0000018
:0117D1000017
:0B17D200436F756E74646F776E3A0011
:0217DD003C00CE
:1017DF00456E746572206E657720636F64653A009D
:0117EF0000F9
:1017F0004C696D697420726561636865642E2E00A2
:0118000000E7
:0C18010031207475726E206C65667400F6
:0D180D0033207475726E73206C6566740074
:0D181A0032207475726E73206C6566740068
:021827000000BF
:041829003230310028
:10182D003E57726F6E672070696E636F64653C0022
:02183D000000A9
:01183F0000A8
:0B18400042757A7A6572204F666600E0
:020000040030CA
:0E00000000081F1EFF8381FF0FC00FE00F409E
:00000001FF
